:03000000020121D9
:03000300C2A8325E
:04000B0012094B3259
:03001300C2AA324C
:03001B00C2AB3243
:0500230012098A3232CF
:100080002A2A2A2A2A2A2A2A2A2A2A2A2A2A2A2AD0
:100090002A20204E455054554E4520494920202ABB
:1000A0002A2056657273696F6E20312E3130202AF6
:1000B0002A20202020202020202020202020202A2C
:1000C0002A2050726F6772616D6564206279202A00
:1000D0002A204D61726B7573204D65696572202A07
:1000E0002A20666F7220537065637472616C202AD7
:1000F0002A20417564696F20202020202020202A9A
:100100002A20284329313939382D32303130202AFC
:100110002A2A2A2A2A2A2A2A2A2A2A2A2A2A2A2A3F
:0101200003DB
:10012100C2AF75D000740078FFF6D8FD7581D07527
:10013100B0FFC0D07450F534F5357410F532F53395
:10014100758921758DFFD28E759852C200D0D0125B
:100151000A6BD28CD2ACD2AFD2A9753000753124E2
:10016100753E00754B0C75420175437F75450075F1
:10017100447F7548007549FF752F01754C31120C8C
:10018100E5120A7AA2939209C2B27EFF7FFFDFFED7
:10019100DEFAD2B2C2957E967FFFDFFEDEFAD295FD
:1001A1007E967FFFDFFEDEFA1201DE12087F7540C8
:1001B100407541001208C775F00174001207D4752B
:1001C100F00274001207D475F00474FF1207D4D240
:1001D100B5C2951201F940FB1201DE80F6300B1316
:1001E100C20B200107D20112087F8007C201120849
:1001F1007F800022D0D0C322C0D01209FF50F5F574
:10020100F030F72AE5F0B4F80302029450FBE5F070
:1002110054F0F539E5F0B4F0030202285009E5F095
:10022100540FF53E02022CE5F0F539E4F53AE539D3
:10023100B480061202F70202CCB490061202D00278
:1002410002CCB4A0030202CCB4B0061203520202E3
:10025100CCB4C00612045D0202CCB4D0061206541E
:100261000202CCB4E00612031A0202CCB4F003027B
:1002710002CCB4F1030202CCB4F2030202CCB4F317
:10028100030202CCB4F6030202CCB4F7030202CC9F
:100291000202CCB4F815052FE52FB54C2EC2967588
:1002A1002F017F40DFFED2960202CCB4FA03020294
:1002B100CCB4FB030202CCB4FC030202CCB4FE03B7
:1002C1000202CCB4FF05E5F00202CCD0D0D322E586
:1002D1003AB40006053A85F03B22B40109053AE536
:1002E100F0547FF53C22753A01E5F0602085F03D40
:1002F100D20212067022E53AB40006053A85F03BB7
:1003010022B40109053AE5F0547FF53C22753A0122
:1003110085F03DC20212067022E53AB40006053AA4
:1003210085F03B22B40109053AE5F0547FF53C2202
:10033100753A0185F03DE53EB53015853D40120821
:10034100C7E53FC0F075F0011207D4D0F01207D312
:1003510022E53AB40006053A85F03B22B4010905CD
:100361003AE5F0547FF53C22753A0185F03D1207DC
:10037100D3E53EB5300280030203F8300105E53CC8
:10038100F54222E53CB47B16E53DB4000280030250
:1003910003F8120A7A12087F754E00D2B222B444D1
:1003A1000FE53DB43F0280025003D20522C205226F
:1003B100B44012E53D700BC20712087B40031208DE
:1003C1007F22D20722B4410EE53D7005C2B5D29518
:1003D10022D2B5C295227402B53C0CE54513E53D28
:1003E10033F545120809227401B53C0CE54413E5C7
:1003F1003D33F54412080922E53CB4210C853DF05A
:10040100A2F6E54492E0F54422B4220C853DF0A227
:10041100F6E54592E0F54522B41005E53DF54B22A0
:10042100B41138E53DB40106754C61020459B402BA
:1004310006754C31020459B40406754C190204596D
:10044100B40806754C0D020459B41006754C070228
:100451000459B42006754C04752F0122E53AB40005
:1004610006053A85F03B22753A0185F03C753DFF62
:100471001207D3E53EB530028003020653E53CB4D2
:1004810000028000B401028000B40025C2041208F9
:0E049100093001028003020653A204C083C09A
:10049F0082E492E0900002120DA1D082D083C201BB
:1004AF00D2B222B40125D20412080930010280030E
:1004BF00020653A204C083C082E492E090000212AD
:1004CF000DA1D082D083C201D2B222B40422C205C0
:1004DF003001028003020653A205C083C082E4925A
:1004EF00E0900003120DA1D082D083C201D2B222BC
:1004FF00B40522D2053001028003020653A205C0C3
:10050F0083C082E492E0900003120DA1D082D083C9
:10051F00C201D2B222B40822C20D300102800302FE
:10052F000653A20DC083C082E492E0900004120D26
:10053F00A1D082D083C201D2B222B40922D20D300F
:10054F0001028003020653A20DC083C082E492E031
:10055F00900004120DA1D082D083C201D2B222B476
:10056F000222C2773001028003020653A277C083B2
:10057F00C082E492E0900007120DA1D082D083C216
:10058F0001D2B222B40322D27730010280030206D5
:10059F0053A277C083C082E492E0900007120DA1AE
:1005AF00D082D083C201D2B222B40622C2763001E9
:1005BF00028003020653A276C083C082E492E090C9
:1005CF000006120DA1D082D083C201D2B222B4078D
:1005DF0022D2763001028003020653A276C083C076
:1005EF0082E492E0900006120DA1D082D083C20166
:1005FF00D2B222B40A1875480030010280030206F5
:10060F0053E548900005120DA1C201D2B222B40BDE
:10061F00187548013001028003020653E548900027
:10062F0005120DA1C201D2B222B40C1875480230C6
:10063F0001028003020653E548900005120DA1C286
:10064F0001D2B22222E53EB53016E53AB4000305D9
:10065F003A22B4010BE5F0547FC333F54D1208096C
:10066F002230011B853C31853E30E531900001126F
:10067F000DA1E530900000120DA1C201D2B222E50A
:10068F003EB53002800122300202800302075C0572
:10069F004EE548B400030206BBB401030206FEB4E4
:1006AF0002030206FEB4030302072922E53C1208E7
:1006BF00965035120AD0500A853CF0B5F0028029C9
:1006CF005027E53C120AAE500CE53FC0F075F00123
:1006DF001207D4D0F030050B12087F7E027FFFDFA8
:1006EF00FEDEFAC2B212080122E53C120AAE22E582
:1006FF003C1208965022853C49E53FC0F075F00149
:10070F001207D4D0F030050B12087F7E027FFFDF77
:10071F00FEDEFAC2B21208012222E53C1208965000
:10072F0027E549B4FF23853C49E53FC0F075F0014B
:10073F001207D4D0F030050B12087F7E027FFFDF47
:10074F00FEDEFAC2B2120801221207D322E54E14BE
:10075F00B4FF01E4F54EE548B40003020780B4018D
:10076F00030207B2B402030207BBB403030207C3B9
:10077F0022120AD05029F536E53C120A8D501F126D
:10078F000AD0501BB536030207AD120896500FE57D
:10079F003FC0F075F0011207D4D0F00206E4221228
:1007AF00087F22E549B53C0312087F22E54E70030E
:1007BF0012087F22E549B53C0712087F7549FF22D1
:1007CF001207D32222CFC0E0CFC0E0C291E5F07F65
:1007DF000833929000D29200C292DFF57F08D0E0EA
:1007EF0033929000D29200C292DFF5D291CFD0E037
:1007FF00CF22C20812088D853D43C0F0E545300475
:0E080F001FC0E0E543300D0DB44002800250E2
:10081D0004E5438002747F23F5F0D0E025F050020B
:10082D0074FF307706254D500274FFF54775F002C1
:10083D001207D4D0F0C0F0E54430031BC0E0E5430F
:10084D00300C0DB4400280025004E5438002747FE9
:10085D0023F5F0D0E0800375F0FF307606254D507E
:10086D000274FFF54675F0041207D4D0F022A208E9
:10087D00B322200708D208D2B212088D22D2082244
:10088D00A208300901B392B322C0E0E531F5372457
:10089D003CF538D0E0C0E0120AF24004D0E0C322AB
:1008AD00D0E0C39531C0F0F5F09001207400932590
:1008BD00F0D0F0F5411208C7D322E5411208CFF56B
:1008CD003F22F536E540B44000403CE54B75F00164
:1008DD0084C5F0E540C39440040404A4C5F0253656
:1008ED00500574FF02094AA2F733A2F63350027481
:1008FD00FFC0E0E540B44005D0E002094AD0E0B4C5
:10090D00FF0274FF02094AE54B75F00184C5F074CE
:10091D003FC39540040404A4C0F0F5F07400C395E2
:10092D00F0C5F0D0E0C53695365005740002094A81
:10093D00A2F733A2F633500274FE02094A22C2A96D
:10094D00C0D0C0E0120A71D2B4A2B44012200A166F
:10095D00D20A200105754A018017754A01801230AF
:10096D000A0FC20A800BE54A6007B40102D20B15CB
:10097D004A300102B2B2D0E0D0D0D2A922C2ACC06E
:10098D00D0C0E0C0F0E9C0E020980A20993AC298A2
:10099D00C2990209F2E53404B4C80274508535F0E9
:1009AD00B5F007E599C2980209D2F534A934A79993
:1009BD00C298E548B40300200004D200D2993099C2
:1009CD00FD8799C2990209F28532F0E533B5F0073A
:1009DD00C200C2990209F204B420027410F533A9C1
:1009ED00338799C299D0E0A9E0D0F0D0E0D0D0D231
:1009FD00AC22C0F0C0D089F0C0F08534F0E535B53B
:100A0D00F00CD0F0A9F0D0D0D0F074F9C322C2AC64
:100A1D0004B4C8027450F535A935E7D2ACD0F0A9AD
:100A2D00F0D0D0D0F0D322C0F0C0D089F0C0F0C04B
:100A3D00E0E53204B4200274108533F0B5F0030202
:100A4D000A3EC2ACF532A932D0E0F7200004D20044
:100A5D00D299D0F0A9F0D0D0D0F0D3D2AC22538916
:100A6D00F0438901758A00758C00D28C22C0E0E8B4
:100A7D00C0E07808760008B810FAD0E0F8D0E0228F
:100A8D00C0F088F0C0F0F5F0C2067808E6B5F004C5
:100A9D007600D20608B810F4D0F0A8F0D0F0A20677
:100AAD0022C0F088F0C0F0F5F0C2067808E67006B6
:100ABD00A6F0D206800408B810F3D0F0A8F0D0F05C
:100ACD00A20622E8C0E075F000C2067808E6B5F08F
:100ADD000280064004F5F0D20608B810F0D0E0F818
:100AED00E5F0A20622B5370280024009B538028032
:100AFD00025002D322C322C0077507083392B612E3
:100B0D000B83D507F7D2B6D2B7000000000020B690
:100B1D0007C2B77400D00722C2B77401D00722C034
:100B2D0007C0E0D2B6E4C2B7750708D2B70000001F
:100B3D000000A2B633C2B70000000000D507ECF5E7
:100B4D0007D0E07004D2B68002C2B6120B83D2B6C3
:100B5D00E507D00722C2B7D2B6D2B7000000000019
:100B6D00C2B60000000000C2B722C2B6D2B7000064
:100B7D00000000D2B622D2B70000000000C2B7229A
:0E0B8D00D20E90007F120C5D5003740122C244
:100B9B000E9007FF120C5D50037410229003FF128E
:100BAB000C5D50037408229001FF120C5D5003740E
:100BBB0004229000FF120C5D500374022290007F00
:100BCB00120C5D5003740122740022C0E0C082C07D
:100BDB0083120B62300E0BD0E0D0E02354FE4400A6
:100BEB00800ED0E023540E44A0120B047013D0E0FF
:100BFB00120B04700ED0E0120B047009120B77D39A
:100C0B0022D0F0D0E0120B77C322C082C083120B2C
:100C1B0062D0E023540E44A0120B0470E4D0E01217
:100C2B000B0470E1E608120B047009D9F7120B776D
:100C3B00D322D0F0120B77C322120B6274A1120BCA
:100C4B0004700A7400120B2C120B77D322120B7741
:100C5B00C322C082C083120B62300E0BD0E0D0E0F7
:100C6B002354FE4401801DD0E023540E44A0120BEC
:100C7B00047020D0E0120B04701B120B62E583236F
:100C8B00540E44A1120B04700C7400120B2C120B9B
:100C9B0077D322D0F0120B77C322C082C083120B02
:100CAB0062D0E023540E44A0120B04701FD0E0124C
:100CBB000B04701A120B6274A1120B047010E9145E
:100CCB00120B2CF608D9F7120B77D322D0F0120B9C
:100CDB0077C322C20FC210020D9A120B8D60F4D291
:100CEB000FD21020B403020D4890000A120DBEB4AF
:100CFB00554B900003120DBEA2E09205900002121C
:100D0B000DBEA2E09204900004120DBEA2E0920D63
:100D1B00900006120DBEA2E09276900007120DBE57
:100D2B00A2E09277900000120DBEF53090000112F8
:100D3B000DBEF531900005120DBEF548227455908D
:100D4B00000A120DA1A20592E0900003120DA1A2C0
:100D5B000492E0900002120DA1A20D92E09000040B
:100D6B00120DA1A27692E0900006120DA1A277922D
:100D7B00E0900007120DA1E530900000120DA1E5E7
:100D8B0031900001120DA1E548900005120DA1C292
:100D9B00B2D2B5C29522C083C082300F11C0E0C061
:100DAB0083C082120BD6D082D083D0E050EFD0829A
:100DBB00D08322C083C082300F0DC083C082120C3F
:0C0DCB005DD082D08350F3D082D0832210
:00000001FF
